:020000040800F2
:1000000000200020E5020008EB020008EF020008D3
:10001000E9130008F5130008D113000800000000E0
:10002000000000000000000000000000DD130008D8
:100030000114000800000000C5130008FD170008A7
:10004000110400081104000811040008110400083C
:10005000110400081104000811040008110400082C
:10006000110400081104000811040008110400081C
:10007000110400081104000811040008110400080C
:100080001104000811040008110400080000000019
:100090000000000000000000000000001104000843
:1000A00011040008110400081104000811040008DC
:1000B000E50F0008B5080008110400081104000845
:1000C00011040008110400081104000811040008BC
:1000D000110400084510000811040008110400086C
:1000E00011040008110400081104000800000000B9
:1000F0000000000000000000000000000000000000
:1001000000000000000000000000000000000000EF
:1001100000000000000000001104000811040008A5
:1001200000000000000000000000000000000000CF
:1001300000000000000000000000000000000000BF
:1001400000000000000000000000000000000000AF
:10015000000000000000000000000000000000009F
:10016000000000000000000000000000000000008F
:10017000000000000000000000000000000000007F
:10018000000000000000000000000000000000006F
:10019000000000000000000000000000000000005F
:1001A000000000000000000000000000000000004F
:1001B000000000000000000000000000000000003F
:1001C0000000000000000000000000005FF808F1DF
:1001D00000B583B000F0AEF9304B314A1360314ABC
:1001E0001360314B314A03E052F8041B43F8041BFF
:1001F0002F498B42F8D32A4B1A682E4B9A4200D0D3
:10020000FEE7284B1A682C4B9A42F9D1234B2B4A14
:1002100013602B4A13602B4B02E0002243F8042B9F
:10022000294A9342F9D3254B1B6813B9244B1B6809
:1002300003B1FEE700F08AF9694601A800F024F94D
:10024000224C234BE41AA410002504E0204B53F861
:10025000253098470135AC42F8DC1E4C1E4BE41AA1
:10026000A410002504E01C4B53F8253098470135B5
:10027000AC42F8DC0099019802F078F80546174C7A
:10028000174BE41AA41004E0013C154B53F824303A
:100290009847002CF8DC284600F0D2F8BABADECA3B
:1002A0000000002010020020000000203064000840
:1002B000140200207856341232547698140200202A
:1002C0009C08002014020020A00800203C04000824
:1002D0003C0400083C0400083C0400083C040008FE
:1002E0003C04000808B5FFF773FF00BEFEE71EF0F0
:1002F000040F0CBFEFF30880EFF309807146414A09
:1003000010472DE9F04182B004460D46124B5F6B59
:10031000D3F838809E6A1B6B13F0020F03D00E4B8C
:10032000DB6A002B0BDB0D4800F0B6F80095434666
:100330003A463146204600F00DF900BEFEE74BF686
:10034000AB6100F081F90028EDD0034B4FF0004283
:10035000DA6202B0BDE8F08100ED00E0905F0008D5
:1003600000BEFEE71EF0040F0CBFEFF30880EFF3B2
:1003700009807146244A10472DE9F04182B00446B5
:100380000D46084B5F6BD3F838809E6A064800F034
:1003900083F8009543463A463146204600F0DAF8A5
:1003A00000BEFEE700ED00E0A05F00081EF0040FB5
:1003B0000CBFEFF30880EFF309807146134A104732
:1003C0002DE9F04182B004460D46084B5F6BD3F82F
:1003D00038809E6A064800F05FF8009543463A462A
:1003E0003146204600F0B6F800BEFEE700ED00E022
:1003F000AC5F000800BEFEE700BEFEE700BEFEE701
:10040000704700000303000879030008C1030008D7
:0404100000BEFEE745
:10041400306400080000002014020020306400084A
:10042400000000000000000014020020A0080020CA
:080434000000000000000000C0
:10044000FEE7000008B503460C4A12685AB10B4A91
:100450001068033323F003030344094A934206D888
:10046000064A136008BD054A06491160EFE703F02C
:1004700015F80C2303604FF0FF30F3E7180200205B
:10048000001C0020A008002001230360014B0B602A
:10049000704700BF040000200FB400B583B004AB68
:1004A00053F8042B01938021074803F085FC0028B2
:1004B00004DC03B05DF804EB04B070470146024869
:1004C00000F034F8F5E700BF200200202DE9F043EA
:1004D00085B004460F46435633BB042528462146C3
:1004E000ABBE0446384605B0BDE8F08314F9010BF5
:1004F00004AA1A4402F8100C0133AB42F6D304AA42
:100500001344002203F8102C4FF00408E94640463B
:100510004946ABBE8046761B002EE3D03546102EF2
:1005200028BF10250023E8E70E46F5E708B5FFF7DA
:10053000CDFF08BD08B500F0EBF8024A024B9A6007
:1005400008BD00BF0000000800ED00E008B500F0A5
:1005500009F908BDF8B504460D4617461E4627485A
:10056000FFF79AFF21682648FFF796FF6168254844
:10057000FFF792FFA1682448FFF78EFFE168234848
:10058000FFF78AFF21692248FFF786FF616921484A
:10059000FFF782FFA1692048FFF77EFFE1691F484E
:1005A000FFF77AFF1E48FFF777FF29461D48FFF740
:1005B00073FF1D4CE16A1D48FFF76EFF216B1C485D
:1005C000FFF76AFFE16B1B48FFF766FF15F0800F2E
:1005D0000AD115F4004F0CD11748FFF75DFF0699BB
:1005E0001648FFF759FFF8BD39461548FFF754FF85
:1005F000EFE731461348FFF74FFFEDE7745E000861
:10060000845E0008945E0008A45E0008B45E0008E2
:10061000C45E0008D45E0008E45E0008F45E0008D2
:10062000045F0008105F000800ED00E0205F000894
:10063000305F0008405F0008705F0008785F0008C6
:10064000505F0008605F000883691A888A4201D001
:10065000002070470268033A012A01D90020704740
:10066000023383610120704782B00023019300931D
:10067000244A136843F480331360224B1B6803F44D
:1006800000330093019B01330193009B1BB9019B35
:10069000B3F5A06FF1D11B4B1B6813F4003F06D0DC
:1006A00001230093009B012B04D002B0704700236C
:1006B0000093F7E7134B5A685A605A685A605A68B1
:1006C0005A605A6822F47C125A605A6842F49812AE
:1006D0005A601A6842F080721A600A4B1B6813F065
:1006E000007FFAD0074B5A6822F003025A605A681A
:1006F00042F002025A60034B5B6803F00C03082BC4
:10070000F9D1D2E70010024008B5FFF7ADFF08BDF0
:1007100008B5114B1A6842F001021A6059680F4A75
:100720000A405A601A6822F0847222F480321A60F9
:100730001A6822F480221A605A6822F4FE025A6073
:100740004FF41F029A600022DA62FFF7DDFF044BCC
:100750004FF000629A6008BD001002400000FFF8F0
:1007600000ED00E01D4B5B6803F00C03042B15D07B
:10077000082B17D01BB11A4B1A4A1A6002E0184B0B
:10078000184A1A60154B5B68C3F30313164AD35C0F
:10079000DAB213490B68D3400B607047104B134A11
:1007A0001A60EFE70D4A53685268C3F3834302337C
:1007B00012F4803F05D10E4A02FB03F3084A13608E
:1007C000E0E7064AD26A02F00F0201320749B1FBA4
:1007D000F2F203FB02F3024A1360D3E70010024077
:1007E0001C00002000127A000C0000200024F400FD
:1007F00000093D0010B40446002002460CE0400809
:100800000133072B07DC10F0010FF8D0400880F00F
:100810008C00C0B2F4E70132A24203DA8B5C58408C
:100820000023EEE710BC7047174A136801331360CA
:10083000154B1B68154A11688B420ADAAC2202FB81
:1008400003F213488258012A03D001330E4A136081
:10085000EEE78B4216DB0C4B00221A600A4B1B683A
:1008600099420ADDAC2202FB03F209488258012AB0
:1008700003D00133044A1360F0E7994202DC024BD3
:1008800000221A60704700BFB00200202400002040
:100890003C03002005490B68054A82FB03021A4409
:1008A000DB17C3EBA2030B60704700BFF802002008
:1008B0009324499270B582B0964A138A9BB223F072
:1008C00001039BB21382944B1B68002B40F0B28053
:1008D000924B1B68002B00F0F280914B1B68012BA0
:1008E00000F0B980022B40F09D808E4B1A6802F018
:1008F00001038D490B60002B40F09E808B4B1968E3
:100900008B4B19608B4B1968AC2303FB01F36833E5
:1009100089490B44043389490B6089490B680133C9
:100920000B6052107F490A607B4A01211160072B3E
:1009300002DD7A4B00221A60764B01229A85814BA8
:1009400000221A606EE0236823EA060626607D4ACC
:10095000136801331360764A126893425ADA002D05
:1009600060D0784B1B6803EB4303744A116801EBBA
:10097000830251F8233054689668072B02D99AB243
:1009800064498A85072B3DD801A252F823F000BFA5
:1009900047090008050A0008B1090008050A00080F
:1009A000BB090008CD090008E1090008F1090008A9
:1009B00023681E40644B1E60C9E7236823EA0606CD
:1009C0002660544B41229A850025C0E723683343B3
:1009D0002360FFF75FFF236823EA06062660B6E779
:1009E00023681E4326604B4B7D229A850025AEE787
:1009F000FFF750FF23681E40534B1E60454B4622B5
:100A00009A85A4E79BB2434A938523681E432660D8
:100A100000259CE73F4B01229A8500233E4A136044
:100A2000484A13603B4A13889BB243F00903138082
:100A300002B070BD012592E7444B19683C4B196028
:100A40003C4B1968AC2303FB01F348333A490B4490
:100A50003A490B6061E7304B01221A603A4B1B6840
:100A600023B13B4A136843F080031360344A136890
:100A700001331360072B1ADD00201060354A13681C
:100A800033490D68344CE554086001331360334A30
:100A9000106883420FDB21460138FFF7ABFE304B75
:100AA000187000231D4A13601B4A136003E0284A94
:100AB00013685B101360174B0F229A85B2E7154B32
:100AC0004FF4FA729A85274B1B680F2B5DD8DFE82D
:100AD00013F010004B0079008D00F00002011A01A4
:100AE0002B01AB00C800E000CB014E016001950175
:100AF000B401084B4CF250329A850E4B1B680E4ADB
:100B0000AC2101FB03235B68012B3ED0154B032274
:100B10001A603AE000040040A8020020A002002071
:100B2000A402002004030020FC0200200003002097
:100B300008060020B00200203C030020FC05002035
:100B400024030020AC0200200C0300200803002036
:100B50000C060020000600201003002020030020C7
:100B60003403002020000020944B1A68944B1A6034
:100B7000944B1A68AC2303FB02F31833924A1344D4
:100B8000924A1360924B01221A60924A1368013311
:100B900013608C4A11688C48AC2202FB0102526837
:100BA000012A02D0042B00F0D6818A4B1B680F2B40
:100BB0007FF738AF874B00221A60874B44F62062DC
:100BC0009A852FE7854B1B681BB1824B0A221A605E
:100BD000DBE7834B33221A60824B02221A60824B7E
:100BE00000221A60814B01221A60CEE701227D4B60
:100BF0001A60724B1968724B1960724B1968AC23FA
:100C000003FB01F3183370490B4470490B60002358
:100C100077490B6077490820086073490B60734B74
:100C20001A606B4B1A60B0E7644B1A68644B1A6029
:100C3000644B1A68AC2303FB02F202F11801624B09
:100C40001944624801601344D3F8A0200132C3F86C
:100C5000A0205F4B01221A605F4B4FF47A629A85A5
:100C600093E75E4B1B681BB15A4B0A221A608CE754
:100C70005B4BCC221A605B4B02221A605A4B00225B
:100C80001A605A4B01221A60534B4FF4FA629A854C
:100C90007BE7534B44221A60524B02221A60524B9C
:100CA00000221A60514B01221A604A4B0A221A6034
:100CB0006BE7424B1A68424B1A60424B1A68AC23EE
:100CC00003FB02F31833404A1344404A1360404B7D
:100CD00001221A6059E7414B1B681BB13D4B0A22A8
:100CE0001A6052E73E4BCC221A603E4B02221A6039
:100CF0003D4B00221A603D4B01221A60364B4FF4E7
:100D0000FA729A8541E7364BBE221A60354B0222B1
:100D10001A60354B00221A60344B01221A602E4BA8
:100D20004FF4FA729A8530E701222E4B1A60324B4B
:100D30001968234B1960234B1968AC2303FB01F39B
:100D4000803321490B44043320490B600023284998
:100D50000B6028490920086023490B60234B1A6067
:100D60001B4B1A601C4B4FF4FA729A850DE7134B1C
:100D70001A68134B1A60134B1A68AC2303FB02F377
:100D80001833114A1344114A1360114B01221A609F
:100D9000FBE6124B1B681BB10E4B0A221A60F4E6ED
:100DA0000F4B33221A600F4B02221A600E4B0022A7
:100DB0001A600E4B01221A60E7E600BF2C030020E8
:100DC00008060020B00200203C030020FC050020A3
:100DD000A802002020000020000400400C03002096
:100DE00004030020A402002024030020A00200200D
:100DF0000006002020030020F40200200122624BA4
:100E00001A60624B1968624B1960624B1968AC2317
:100E100003FB01F3803360490B4404335F490B60EB
:100E200000235F490B605F49082008605E490B6042
:100E30005E4B1A605E4B1A60A7E65E4BDA795E4B3A
:100E40001B789A4202D0FFF7EFFC9EE604225B4932
:100E50000DEB020002F028FB019B5A1E12F1030F5A
:100E6000F1D8574A1360EEE74A4B1B684A4AAC2157
:100E700001FB03230022C3F8A8204E4B1A7A4E4BE5
:100E80001B789A4212D0FFF7CFFC4E4B10221A600B
:100E9000404B1B68404AAC2101FB03235B68012BDC
:100EA0007FF473AE474B0B221A606EE6042243496F
:100EB0000DEB020002F0F8FA019B013B13F1030F66
:100EC00037D8414B414A13603A4A11781970527829
:100ED0005A70B3F90030C3EB431203EB8202531094
:100EE0003B49B1EB620F2DD03A4A93422ADB3A4A92
:100EF000934227DC274A1268384941F822302648B5
:100F0000AC2101FB0201D1F8A4000130C1F8A4001A
:100F10000120C1F8A80003F55643D83330498B426D
:100F200010D91D4BAC2101FB02320023C2F8A830BE
:100F300008E0184B1B68184AAC2101FB0323002270
:100F4000C3F8A8201C4BFF221A700A22002119485E
:100F500002F0B8FA97E7AC2202FB0102D2F89C300B
:100F6000013BC2F89C30002B07DC0B4BAC2202FB90
:100F700001310423C1F89C3017E6FFF755FC114BF3
:100F800010221A6011E600BFA4020020F402002023
:100F900008060020B00200203C030020FC050020D1
:100FA000000600202003002024030020A0020020CF
:100FB000A8020020100300203403002011030020A9
:100FC0000406002020000020280300203803002011
:100FD000084C01002929FFFF47E80100EC0500202B
:100FE00020BF02004FF080431B8A13F0010F1BD07B
:100FF000104B1B784BB10F4A1378013BDBB21370D7
:10100000137813B90C4B01221A700C4B1B785BB18F
:101010000A4A1378013BDBB21370137823B9084AEC
:10102000D36823F48053D3604FF0804300221A82A8
:10103000704700BFB4020020B6020020B5020020B5
:10104000000801403B4B1B8813F0400F21D03A4A67
:101050001378DBB23949585C36490B889BB223F0D0
:1010600040039BB20B801378DBB2354A126893427F
:1010700036DA344AD36843F48053D36080B2888030
:101080002D4A13780133DBB213701378DBB2FF2BD8
:101090003CD0284B1B8813F0200F1DD02A4B1B7807
:1010A00013B9294B01221A70284B04221A70284BBD
:1010B00000221A701F4A13889BB223F020039BB2B0
:1010C00013809088234A1378DBB22349C8541378DD
:1010D0000133DBB213701378164B00221A8070476D
:1010E000144A93899BB243F02003938193899BB266
:1010F00023F040039BB29381A2F54052D36823F4BE
:101100008053D360154B00221A70B9E700220A4BB6
:101110001A700C49CB6823F48053CB6001F5405121
:101120008B899BB223F040039BB28B810B4B1A70CF
:10113000AFE700BF00380140C102002010060020C8
:10114000BC02002000080140B7020020B4020020C9
:10115000B6020020C002002010070020B8020020C4
:10116000154B1B78DBB2012B24D0144B18600330D5
:10117000C0B2134B1870134B1A8892B222F040027F
:1011800092B21A809A8992B242F040029A819A8968
:1011900092B222F0200292B29A810B49CA6842F4BC
:1011A0008052CA60094A12789A800123024A137059
:1011B000074A1370704700BFB8020020BC0200202D
:1011C000B502002000380140000801401006002050
:1011D000C102002035498A8902F400528B899BB2F2
:1011E00023F400539BB28B81314B1B68013B072BCF
:1011F0000DD8DFE803F0041B242D363F48512D4B5A
:101200001B682D49A1FB03131B0A2C490B602B4BB8
:101210001B684FF6F0711940C3F342030B43234997
:101220000B818B899BB21A438A817047214B1B68C3
:101230002149A1FB03135B0A20490B60E7E71D4B23
:101240001B681D49A1FB03139B0A1C490B60DEE7C9
:10125000184B1B681849A1FB0313DB0A17490B60E5
:10126000D5E7144B1B681449A1FB03131B0B13494F
:101270000B60CCE70F4B1B681149A1FB0313DB0B81
:101280000E490B60C3E70B4B1B680D49A1FB031311
:101290001B0C0A490B60BAE7064B1B680849A1FB07
:1012A00003135B0C05490B60B1E700BF0038014038
:1012B000280000201C000020B5814E1B580800208B
:1012C000C5B3A29130B4FF2214464D1E51B110F89F
:1012D000013B63400549CC5C5440054AD256D2B22A
:1012E0002946F2E742EA042030BC7047BC5F0008A0
:1012F000BC60000800687047034BDB6813F0010F07
:101300000CBF0120002070470020024008B5054BAB
:10131000054A5A6002F188325A60FFF7EDFF002853
:10132000FBD008BD0020024023016745024A136933
:1013300043F08003136170470020024008B50A4B58
:101340001A6942F002021A6158611A6942F04002B9
:101350001A61FFF7D1FF0028FBD0034A136923F07D
:101360000203136108BD00BF0020024038B50546E6
:101370000C460D4A136943F001031361FFF7BCFFEC
:101380000028FBD0A3B22B80FFF7B6FF0028FBD0CC
:10139000240C6C80FFF7B0FF0028FBD0024A1369D1
:1013A00023F00103136138BD0020024038B5044624
:1013B0000D46FFF7ABFF29462046FFF7D7FFFFF7A3
:1013C000B5FF38BD4EF27C234FF080421A60704763
:1013D0004EF27C234FF480021A6070474EF27C2359
:1013E0004FF000621A6070474EF27C234FF4801277
:1013F0001A6070474EF27C234FF400121A60704757
:101400004EF27C234FF080521A60704708B5654851
:10141000FFF770FFC0B2644B1870FF2800F08580A2
:101420006248FFF767FFC0B2614B1860FF287FD0AA
:101430006048FFF75FFF604B1860B0F1FF3F7AD064
:101440005E48FFF757FF5C4B5860B0F1FF3F75D027
:101450005B48FFF74FFF584B9860B0F1FF3F70D0EB
:101460005848FFF747FF544BD860B0F1FF3F6BD0AF
:101470005548FFF73FFF554B1860B0F1FF3F66D06E
:101480005348FFF737FF514B5860B0F1FF3F62D030
:101490005048FFF72FFF4D4B9860B0F1FF3F5ED0F3
:1014A0004D48FFF727FF494BD860B0F1FF3F5AD0B6
:1014B0004A48FFF71FFF80B2494B18804FF6FF7371
:1014C000984254D04748FFF715FF80B2464B18802A
:1014D0004FF6FF7398424ED04448FFF70BFF80B29F
:1014E000434B18804FF6FF73984248D04148FFF7AE
:1014F00001FF80B2404B18804FF6FF73984243D0F3
:101500003E48FFF7F7FE80B23D4B18804FF6FF7361
:1015100098423ED03B48FFF7EDFE80B23A4B188030
:101520004FF6FF73984238D008BD1C221A7077E737
:1015300003221A607CE700221A6081E700225A60C9
:1015400086E700229A608BE70022DA6090E740F697
:10155000FF721A6094E740F6FF725A6098E740F60F
:10156000FF729A609CE740F6FF72DA60A0E71C4BBE
:101570001E221A80A6E71C4BF0221A80ACE71C4BF7
:101580004FF496721A80B1E71B4B4FF4E1621A8058
:10159000B6E71B4B01221A80BCE71B4B04221A80C2
:1015A000C2E700BF00B800085008002004B80008D7
:1015B0002800002008B80008100800200CB8000817
:1015C00010B8000814B8000818B800082408002053
:1015D0001CB8000820B8000824B8000828B8000883
:1015E000880800202CB800088A08002030B80008BD
:1015F0002008002034B800085408002038B800083B
:101600003C0800203CB800085C08002010B5FFF73B
:101610007DFE284C2046FFF791FE274B1978204687
:10162000FFF7C4FE254B19682548FFF7BFFE254C80
:1016300021682548FFF7BAFE61682448FFF7B6FE27
:10164000A1682348FFF7B2FEE1682248FFF7AEFE2B
:10165000214C21682148FFF7A9FE61682048FFF767
:10166000A5FEA1681F48FFF7A1FEE1681E48FFF72D
:101670009DFE1E4B19881E48FFF798FE1D4B1988CA
:101680001D48FFF793FE1D4B19881D48FFF78EFE7E
:101690001C4B19881C48FFF789FE1C4B19881C48F5
:1016A000FFF784FE1B4B19881B48FFF77FFEFFF7EF
:1016B0003DFE10BD00B800085008002028000020A2
:1016C00004B800081008002008B800080CB800088A
:1016D00010B8000814B800082408002018B8000842
:1016E0001CB8000820B8000824B8000888080020AA
:1016F00028B800088A0800202CB80008200800201C
:1017000030B800085408002034B800083C08002015
:1017100038B800085C0800203CB8000838B500F56F
:10172000000000F53C6004012046FFF7E3FD084D92
:101730002860201DFFF7DEFD686004F10800FFF758
:10174000D9FDA86004F10C00FFF7D4FDE86038BDB6
:101750007008002010B500243F2C0BD804F50000C1
:1017600000F53C600001FFF7C5FDB0F1FF3F03D07D
:101770000134F1E74FF0FF34B4F1FF3F09D094B9E1
:101780000C4A0023136053609360D3600A4A1360CD
:1017900010BD3F20FFF7C2FF074B00221A60074B26
:1017A00001221A60F4E7601EFFF7B8FF024B1C60CD
:1017B000EEE700BF700800208C080020D002002057
:1017C00010B5FFF7A3FD00240EE00A4B186800F5E2
:1017D000000000F53C6004EB8000074B53F8241038
:1017E0008000FFF7E3FD0134032CEED9FFF79EFDE7
:1017F00010BD00BF8C080020700800203F4A13680D
:10180000013313603E4B1B68322B05DD0A3B3C4A1B
:1018100013609BB23B4A93873B4B1B680A2B06DD48
:10182000043B394A13609BB2364AA2F84030374B2A
:101830001B88042B00D07047354B9B6813F4004F76
:101840000FD1344B1B68344A126893420CD20133D7
:1018500030490B609A4207D1304A13680133136054
:1018600002E02C4B00221A60294B9B6813F4804F36
:101870000FD1284B5B68284A126893420CD201337F
:1018800024494B609A4207D1244A5368013353607C
:1018900002E0204B00225A601D4B9B6813F4005F4E
:1018A0000FD11C4B9B681C4A126893420CD2013327
:1018B00018498B609A4207D1184A936801339360A4
:1018C00002E0144B00229A60114B9B6813F4805F76
:1018D0000FD1104BDB68104A12689342ABD2013330
:1018E0000C49CB609A42A6D10C4AD3680133D3602D
:1018F0007047084B0022DA609DE700BFE402002039
:101900002C00002000080040300000205C0800206F
:10191000000C0140D40200203C0000207008002090
:1019200082B003888DF80730C3F307238DF80630A3
:10193000BDF8060002B07047002393420DDA30B4C0
:101940005C0001340D5D00F8135011F8135005557B
:1019500001339342F4DB30BC704770470278C74BC9
:101960001B789A4200D0704770B5A2B00446437805
:10197000DA1ED2B2012A06D9053BDBB2012B40F2B6
:101980002D8322B070BD0621FFF79CFCADF804004A
:10199000A01DFFF7C5FFBDF804308342F1D1B84B5D
:1019A0001B68B3F5FA6F03DAB54B4FF4FA621A60AD
:1019B000A01CFFF7B5FF0546201DFFF7B1FF064647
:1019C0008022002102A801F07DFDAE4BAB4A1278C7
:1019D0001A7062785A7072009A70632D00F0B780A6
:1019E0001E2D00F0BA801F2D00F0BD80202D00F0CC
:1019F000C080212D00F0C3803C2D00F0C6803D2D1D
:101A000000F0C9803E2D00F0CC803F2D00F0CF804B
:101A1000642D00F0D280652D00F0D580662D00F099
:101A2000D880672D00F0DB80A02D00F0DE80A12D96
:101A300000F0E180A22D00F0E480A32D00F0E7800B
:101A4000AA2D00F0EA80AB2D00F0ED80AC2D00F067
:101A5000F080AD2D00F0F380962D00F0F680972DEC
:101A600000F0F980982D00F0FC80992D00F0FF80A7
:101A7000462D00F03D81472D00F04C81482D00F0AF
:101A80005B81492D00F06A814A2D00F079814B2D50
:101A900000F088814C2D00F097814D2D00F0A6813B
:101AA000502D00F0B581512D00F0C781522D00F06E
:101AB000D981532D00F0E881C82D00F0FA81C92D9D
:101AC00000F0FD81CA2D00F00082D22D00F00382CB
:101AD000D32D00F00682D42D00F00982D52D00F020
:101AE0000C82DC2D00F00F82DD2D00F01282DE2D45
:101AF00000F01582DF2D00F01882E02D00F01B822F
:101B0000E12D00F01E82FB2D00F02182FC2D00F063
:101B10002482FD2D00F02782FE2D00F02F8276001A
:101B2000594C324602A9204601F0BEFCF51C033C8C
:101B300029462046FFF7C6FBADF80400012201A9A3
:101B40006019FFF7F9FE701DFFF70AFB19E732462F
:101B50004E4902A8FFF7F0FE42E732464C4902A880
:101B6000FFF7EAFE3FE732464A4902A8FFF7E4FEE4
:101B70003CE73246484902A8FFF7DEFE39E7324625
:101B8000464902A8FFF7D8FE36E73246444902A884
:101B9000FFF7D2FE33E73246424902A8FFF7CCFEF8
:101BA00030E73246404902A8FFF7C6FE2DE732462D
:101BB0003E4902A8FFF7C0FE2AE732463C4902A888
:101BC000FFF7BAFE27E732463A4902A8FFF7B4FE0C
:101BD00024E73246384902A8FFF7AEFE21E7324635
:101BE000364902A8FFF7A8FE1EE73246344902A88C
:101BF000FFF7A2FE1BE73246324902A8FFF79CFE20
:101C000018E73246304902A8FFF796FE15E732463C
:101C10002E4902A8FFF790FE12E732462C4902A88F
:101C2000FFF78AFE0FE732462A4902A8FFF784FE33
:101C30000CE73246284902A8FFF77EFE09E7324644
:101C4000264902A8FFF778FE06E73246244902A893
:101C5000FFF772FE03E73246224902A8FFF76CFE47
:101C600000E73246204902A8FFF766FEFDE632464D
:101C70001E4902A8FFF760FEFAE600BF50080020E8
:101C80002C0000201006002013060020E402002093
:101C9000EC050020F0050020F4050020F8050020E8
:101CA0006008002064080020680800206C080020FC
:101CB0007008002074080020780800207C080020AC
:101CC0001008002014080020180800201C0800201C
:101CD00024080020280800202C08002030080020BC
:101CE0008008002082080020840800208608002048
:101CF0000023ADF80630A74B9B6813F0800F02D08D
:101D00000123ADF8063001220DF1060102A8FFF70C
:101D100013FEB0E60023ADF806309E4B9B6813F02F
:101D2000400F02D00123ADF8063001220DF106016B
:101D300002A8FFF701FEA1E60023ADF80630954B9F
:101D40009B6813F0200F02D00123ADF8063001226A
:101D50000DF1060102A8FFF7EFFD92E60023ADF8B2
:101D600006308C4B9B6813F0100F02D00123ADF8A6
:101D7000063001220DF1060102A8FFF7DDFD83E622
:101D80000023ADF80630834B9B6813F4004F02D05C
:101D90000123ADF8063001220DF1060102A8FFF77C
:101DA000CBFD74E60023ADF806307A4B9B6813F444
:101DB000804F02D00123ADF8063001220DF106015B
:101DC00002A8FFF7B9FD65E60023ADF80630714BB8
:101DD0009B6813F4005F02D00123ADF806300122A6
:101DE0000DF1060102A8FFF7A7FD56E60023ADF8A6
:101DF0000630684B9B6813F4805F02D00123ADF876
:101E0000063001220DF1060102A8FFF795FD47E615
:101E10000023ADF8063003F1804303F584339B685B
:101E200013F4006F02D00123ADF8063001220DF14A
:101E3000060102A8FFF780FD35E60023ADF8063065
:101E400003F1804303F584339B6813F4004F02D001
:101E50000123ADF8063001220DF1060102A8FFF7BB
:101E60006BFD23E60023ADF806304A4B9B6813F068
:101E7000080F02D00123ADF8063001220DF1060152
:101E800002A8FFF759FD14E60023ADF8063003F170
:101E9000804303F584339B6813F0020F02D00123C3
:101EA000ADF8063001220DF1060102A8FFF744FD4E
:101EB00002E63246384902A8FFF73EFDFFE532460A
:101EC000364902A8FFF738FDFCE53246344902A83E
:101ED000FFF732FDF9E53246324902A8FFF72CFD43
:101EE000F6E53246304902A8FFF726FDF3E5324613
:101EF0002E4902A8FFF720FDF0E532462C4902A842
:101F0000FFF71AFDEDE532462A4902A8FFF714FD56
:101F1000EAE53246284902A8FFF70EFDE7E532461A
:101F2000264902A8FFF708FDE4E53246244902A845
:101F3000FFF702FDE1E53246224902A8FFF7FCFC6B
:101F4000DEE53246204902A8FFF7F6FCDBE5324623
:101F50001E4902A8FFF7F0FCD8E532461C4902A84A
:101F6000FFF7EAFCD5E51B4B1B88ADF8063032467F
:101F70000DF1060102A8FFF7DFFCCDE5164B1B783B
:101F8000ADF8063032460DF1060102A8FFF7D4FC89
:101F9000C5E500BF000C0140C4020020C8020020BB
:101FA00034000020880800208A0800202008002033
:101FB0005408002052080020400800204208002059
:101FC0004408002046080020480800203C08002063
:101FD0005C08002028000020500800200621FFF7A0
:101FE00071F90546A01DFFF79BFC85427FF4C9AC43
:101FF000894B1A6842F227339A4203DC864B42F23D
:1020000028321A60A01CFFF78BFC0546201DFFF745
:1020100087FC0446814B1A788149824801F044FAD2
:10202000A5F15000AE2800F2EB80DFE810F0AF0021
:10203000BD00CB00D900E900E900E900E900E900B2
:10204000E900E900E900E900E900E900E900E90048
:10205000E900E900E900E700EE00F1000301E90012
:10206000E900E900E900E900E900E900E900E90028
:10207000E900E900E900E900E900E900E900E90018
:10208000E900E900E900E900E900E900E900E90008
:10209000E900E900E900E900E900E900E900E900F8
:1020A000E900E900E900E900E900E900E900E900E8
:1020B000E900E900E900E900E900E900E900E900D8
:1020C000E900E900E900E900E900E900E9000601AA
:1020D0000D0114011B01E900E900E900E900E90034
:1020E000E9002201290130013701E900E900E90096
:1020F000E900E900E900E900E900E900E900E90098
:10210000E900E900E900E900E900E900E900E90087
:10211000E900E900E900E900E900E900E9003E0121
:1021200052015501E900E900E900E900E900E90090
:10213000E90058015D0162016701E900E900E90079
:10214000E900E900E900E900E900E900E900E90047
:10215000E900E900E900E900E900E900E900E90037
:10216000E900E900E900E900E900E900E900E90027
:10217000E900E900E900E900E900E900E900E90017
:10218000E900E9006C01710176017B01012C05D0A9
:10219000254AD36823F40063D36031E0224AD36830
:1021A00043F40063D3602BE0012C05D01E4AD368B2
:1021B00023F40043D36023E01B4AD36843F4004375
:1021C000D3601DE0012C05D0184AD36823F0080322
:1021D000D36015E0154AD36843F00803D3600FE0DD
:1021E000012C05D0104AD36823F00203D36007E026
:1021F0000D4AD36843F00203D36001E00C4B1C602E
:102200000820FEF7ADFFFFF7BCBB094B5C60F7E7AA
:10221000074B9C60F4E700BF2C000020C0020020A8
:10222000100700201006002000080140000C0140AB
:10223000700800203E4BDC60E2E73E4B1A883E4BC4
:102240001A60FFF7E3F9DBE73A4B5A883A4B5A60DA
:10225000FFF7DCF9D4E7374B9A88374B9A60FFF7E2
:10226000D5F9CDE7334BDA88334BDA60FFF7CEF997
:10227000C6E7304B1A88314B1A60FFF7C7F9BFE742
:102280002C4B5A882D4B5A60FFF7C0F9B8E7294B01
:102290009A882A4B9A60FFF7B9F9B1E7254BDA889B
:1022A000264BDA60FFF7B2F9AAE7254B1B8833B952
:1022B000244B1B881BB9244B1B88012B06D0204BB9
:1022C0001B88062B9CD11E4B1C8099E71C4B1C8045
:1022D000F5E71C4B1C8093E71B4B1C8090E71B4BC6
:1022E0001C80FFF793F98BE7194B1C80FFF78EF9E1
:1022F00086E7184B1C80FFF789F981E7164B1C8095
:10230000FFF784F97CE7154B1C80FFF77FF977E72F
:10231000134B1C80FFF77AF972E7124B1C60FFF732
:1023200075F96DE7104B1C70FFF770F968E700BF97
:102330007008002034080020100800202408002025
:10234000C4020020C80200203400002088080020B9
:102350008A08002020080020540800203C080020A3
:102360005C08002028000020500800202DE9F04FD4
:1023700083B0FEF7CDF9AA4A936943F4804343F052
:102380003D039361D36943F00703D361A54B1968FB
:1023900021F003011960196821F00C011960196816
:1023A00021F030011960196821F0C0011960196825
:1023B00021F440311960196821F44021196019682D
:1023C00021F440111960196821F440011960536823
:1023D00023F44043536053685360936943F400739C
:1023E0009361914B9A6842F008029A609A6842F0B1
:1023F00004029A608C4B9B6813F0040FFAD18A4B4D
:102400009A6842F001029A609A6842F400029A6067
:102410009A6842F4F0129A605A6842F480725A60E4
:102420001A6942F007021A615A6B22F01F025A63BE
:102430001A6942F038021A615A6B42F020025A635C
:102440001A6942F4E0421A615A6B42F480525A63AC
:102450001A6942F460321A615A6B42F420325A63AC
:10246000DA6A42F44012DA629A6842F002029A6032
:102470009A6842F480729A6069494B6943F001039B
:102480004B616A4B6A4A9A606A4ADA6004225A606F
:102490001A6842F020021A601A6842F080021A603C
:1024A0001A6842F480621A601A6842F480721A60F4
:1024B0001A6842F001021A605F4A536823F0F00381
:1024C0005360536843F0A0035360536823F00F0335
:1024D0005360536843F00A035360584B188C40F420
:1024E00080501884188C40F480701884032018855C
:1024F00042F20F7098854FF47A74A3F8404040F68A
:10250000B8309887988B40F4D0409883988B40F0EF
:1025100068009883188840F001001880CB6943F068
:102520000203CB61464B07211985998941F00101CE
:1025300099819C85198841F00901198003F582333E
:10254000596841F480515960596821F440415960FB
:102550003C48416841F000714160596841F0805148
:102560005960596821F040415960D96821F400410F
:10257000D960136843F480531360136823F4404315
:102580001360FEF743FF304B1B88042B00F0A28042
:10259000244B5A6822F0F0025A605A6842F0A002B6
:1025A0005A60DA6822F48052DA605A6822F4802293
:1025B0005A605A6842F400325A60DA6882F4007253
:1025C000DA6003F540539A8902F480529A811A8A9C
:1025D00042F400521A829A8942F4005242F00C02EC
:1025E0009A819A8942F020029A81FEF7F3FD0C4A03
:1025F000D36943F00103D36114490B6802F14672B9
:1026000002F5E7328332A2FB03239B0C013B9BB212
:102610004FF080421385938943F00103938117E0C3
:102620000010024000080140002401400800024060
:102630004C24014034080020000C014000080040F8
:1026400000040040000001405C0800201C00002045
:10265000664B18684FF4966303FB00F3644880FBF5
:102660000354DB17C3EBA4139BB29385138843F089
:10267000010313800B68A0FB03239B09013BB3F10B
:10268000807F09D25B4A53605B4BF02183F82310B3
:102690000023936007231360584B19685848FDF7CF
:1026A000FBFE584B4FF080521A6020225A60564A67
:1026B000936843F480039360544B41F658321A6098
:1026C000534B9B6813F0400F07D100230193002464
:1026D000A346BCE0FFF73EF85AE701230193F6E773
:1026E0000C46B4E00C46B2E04A4B1B78002B00F0DD
:1026F000B480494B1B68B3F5FA7F03DA464B4FF4BD
:10270000FA721A60454B1B78DBB2032B0CD8434D91
:102710002A780021424800F0D5FE00232B70414A60
:1027200013703C4A13709DE03D48FFF717F9EEE740
:10273000BBF10F0F02D93C4B1B68C3B9BBF1050FAE
:1027400040F24181394B1B68002B00F03C81304B3B
:102750009B6813F0400F01D1019B9BB92C4B9B68E8
:1027600013F0400F00F02F81012301932BE1FEF7BE
:10277000CDFD2F48FEF7E2FDFEF7D8FD2A4B0022E3
:102780001A60DBE7FFF71CF8284B00221A60E5E728
:102790001F4B9B6813F4006F04D01C4B40F6C4120F
:1027A0001A604EE0194B4FF4FA721A6049E0184B68
:1027B0009B6813F4004F04D0144B40F6C4121A6007
:1027C0003FE0124B4FF4FA721A603AE0194B9B68E3
:1027D00013F0080F04D00D4B40F6C4121A6030E01D
:1027E0000A4B4FF4FA721A602BE000BF5808002021
:1027F000D34D621010E000E000ED00E01C0000206E
:10280000BC61000800E100E000240140300000202D
:1028100000080140B70200202C000020C002002068
:1028200010070020B6020020D0020020380000204F
:1028300000BC0008000C0140AA4B4FF49672A3F8AC
:102840004020A94B1B88022B00F0EB800C46A74BC5
:102850001B78DBB2012B3FF447AFA54AD36823F4C2
:102860008073D360A34AB2F80090A34BC3F80090E2
:1028700057885F6096889E60D588DD609F4B18689A
:1028800000F0A8FB82469E4B186800F0A3FB804630
:102890000146504600F0ECFA8246002100F086FD29
:1028A000A0B9484600F096FB414600F0E1FA00F07E
:1028B000AFFD00B200F092FB514600F097FC914949
:1028C00000F0E0FB00F0CAFD8F4B18808B4B58687E
:1028D00000F080FB81468A4B586800F07BFB804605
:1028E0000146484600F0C4FA8146002100F05EFD32
:1028F000A0B9384600F06EFB414600F0B9FA00F08E
:1029000087FD00B200F06AFB494600F06FFC7D498C
:1029100000F0B8FB00F0A2FD7B4B5880774B986825
:1029200000F058FB8046764B986800F053FB074652
:102930000146404600F09CFA8046002100F036FD3A
:10294000A0B9304600F046FB394600F091FA00F09D
:102950005FFD00B200F042FB414600F047FC6949D0
:1029600000F090FB00F07AFD674B9880634BD868CD
:1029700000F030FB0746624BD86800F02BFB0646A0
:102980000146384600F074FA0746002100F00EFDBB
:10299000A0B9284600F01EFB314600F069FA00F0AD
:1029A00037FD00B200F01AFB394600F01FFC554914
:1029B00000F068FB00F052FD534BD8804A4B1B8857
:1029C000042B3FF4B5AE514B1B68514A12689B1A59
:1029D000B3F57A7FFFF43BAF4C4B1A684C4B1A604F
:1029E0000BF1010B611C4B4A82FB0432E317C3EB72
:1029F000620303EB8303E31A042B3FF622AF01A229
:102A000052F823F091270008AF270008CD270008CF
:102A100039280008192A0008324B0022A3F8402068
:102A20000FE7334A926812F4006F57D00120304A02
:102A3000926812F4806F53D01A46024395B2364A18
:102A40001580364A926812F0040F6BD00120334A89
:102A5000926812F0080F67D01A46024396B22E4AC7
:102A60005680234A926812F0200F5FD00120204A3E
:102A7000926812F0100F5BD01A46024394B2264AB5
:102A800094801B4A926812F4004F53D00120184AD8
:102A9000926812F4804F4FD01A46024392B21E48F9
:102AA000C2801348806810F4005F47D00120104FA7
:102AB000BF6817F4805F00D10023034316480381E9
:102AC00017480088062800F2BD81DFE810F03900C1
:102AD0008D00AB00EC000A014A017F010020A6E74F
:102AE0000022AAE7000800405C080020B60200208F
:102AF000000C014034080020600800202408002059
:102B00001008002000401C4680080020E40200203D
:102B1000CC0200206766666640080020000801407D
:102B2000C4020020002092E7002296E700209EE7E2
:102B30000022A2E70020AAE70022AEE70020B6E7C5
:102B4000964F388800F1010CA7F800C0944F3F88D9
:102B5000B84218D993480088B0B1022D11D0012095
:102B6000012E01D040F00200022C01D040F0040000
:102B7000012A01D040F00800022B05D040F01000DF
:102B800002E00020ECE70020874BDA6842F40062A4
:102B9000DA60DA6822F40042DA6003F58063DA680A
:102BA00022F00802DA609B6813F0400F18D17F4AC8
:102BB000138801339BB213807D4A1288934240F2FE
:102BC00030817C4B1B881BB97B4B1B88012B03D0AE
:102BD000764B00221A8024E1784B01221A80F7E715
:102BE000724B00221A801CE16F4BDA6822F40062FB
:102BF000DA60DA6822F40042DA60714AD36823F0BE
:102C00000803D360654A1388581C1080644A1288F0
:102C1000934240F21981694B02221A8000205F4BD7
:102C20001880FEE05D480088471CBFB2DFF870C125
:102C3000BCF800C0604518D95A480088B0B1012DD1
:102C400011D00120022E01D040F00200022C01D050
:102C500040F00400022A01D040F00800012B05D00A
:102C600040F0100002E00020ECE700204E4BDA6854
:102C700022F40062DA60DA6842F40042DA60504A14
:102C8000D36823F00803D3607A1C444B1A804D4B61
:102C90001B889F4240F2C580484B03221A803F4B5D
:102CA00000221A80BDE0404BDA6822F40062DA604C
:102CB000DA6822F40042DA60414AD36823F008035C
:102CC000D360364A1388581C1080354A12889342C4
:102CD00040F2BC80394B04221A8000202F4B188010
:102CE0009FE02E480088471CBFB2DFF8B4C0BCF894
:102CF00000C0604518D92B480088B0B1022D11D012
:102D00000120012E01D040F00200012C01D040F042
:102D10000400022A01D040F00800022B05D040F048
:102D2000100002E00020ECE700201F4BDA6822F4DC
:102D30000062DA60DA6822F40042DA60204AD3687E
:102D400043F00803D3607A1C144B1A801E4B1B8877
:102D50009F4266D9194B05221A80104B00221A8017
:102D60005FE0114BDA6822F40062DA60DA6822F47C
:102D70000042DA60124AD36823F00803D360074A9E
:102D80001388581C1080064A1288934260D900208C
:102D90000A4B1880014B188043E000BFC602002098
:102DA000880800203C08002000080140C2020020E2
:102DB00054080020C802002034000020C402002073
:102DC000000C01408A080020200800202148C76824
:102DD00027F40067C760C76827F40047C7601E4F25
:102DE000F86820F00800F860013DADB2012D27D948
:102DF0000120013EB6B2012E01D940F00200013C93
:102E0000A4B2012C01D940F00400013A92B2012A87
:102E100001D940F00800013B9BB2012B01D940F0E1
:102E200010000E4B18800E4B1B88002B3FF458AC43
:102E300000283FF457AC0B4B06221A800C4606E5DF
:102E40000020D6E70020ECE70020EAE70020E8E7D2
:102E50000020E6E700080140000C01405208002075
:102E60003C080020C402002080F0004002E000BFC7
:102E700081F0004142001FBF5FEA410392EA030F65
:102E80007FEA226C7FEA236C6AD04FEA1262D2EBAF
:102E90001363C1BFD218414048404140B8BF5B42B4
:102EA000192B88BF704710F0004F40F4000020F04D
:102EB0007F4018BF404211F0004F41F4000121F063
:102EC0007F4118BF494292EA030F3FD0A2F10102AD
:102ED00041FA03FC10EB0C00C3F1200301FA03F1EB
:102EE00000F0004302D5494260EB4000B0F5000F0E
:102EF00013D3B0F1807F06D340084FEA310102F1CD
:102F00000102FE2A51D2B1F1004F40EBC25008BF7E
:102F100020F0010040EA03007047490040EB000048
:102F200010F4000FA2F10102EDD1B0FA80FCACF177
:102F3000080CB2EB0C0200FA0CF0AABF00EBC25076
:102F400052421843BCBFD0401843704792F0000F64
:102F500081F4000106BF80F400000132013BB5E7B7
:102F60004FEA41037FEA226C18BF7FEA236C21D02D
:102F700092EA030F04D092F0000F08BF0846704792
:102F800090EA010F1CBF0020704712F07F4F04D160
:102F9000400028BF40F00040704712F100723CBF73
:102FA00000F50000704700F0004343F0FE4040F49D
:102FB000000070477FEA226216BF08467FEA23635B
:102FC0000146420206BF5FEA412390EA010F40F446
:102FD000800070474FF0000304E000BF10F0004392
:102FE00048BF40425FEA000C08BF704743F0964379
:102FF00001464FF000001CE050EA010208BF704794
:103000004FF000030AE000BF50EA010208BF70471A
:1030100011F0004302D5404261EB41015FEA010C2F
:1030200002BF84460146002043F0B64308BFA3F127
:103030008053A3F50003BCFA8CF2083AA3EBC25309
:1030400010DB01FA02FC634400FA02FCC2F1200228
:10305000BCF1004F20FA02F243EB020008BF20F05F
:103060000100704702F1200201FA02FCC2F12002C5
:1030700050EA4C0021FA02F243EB020008BF20EABA
:10308000DC7070474FF0FF0C1CEAD0521EBF1CEAE8
:10309000D15392EA0C0F93EA0C0F6FD01A4480EAD6
:1030A000010C400218BF5FEA41211ED04FF00063BF
:1030B00043EA501043EA5111A0FB01310CF00040EB
:1030C000B1F5000F3EBF490041EAD3715B0040EA11
:1030D000010062F17F02FD2A1DD8B3F1004F40EBE1
:1030E000C25008BF20F00100704790F0000F0CF0B4
:1030F000004C08BF49024CEA502040EA51207F3A78
:10310000C2BFD2F1FF0340EAC250704740F4000052
:103110004FF00003013A5DDC12F1190FDCBF00F043
:1031200000407047C2F10002410021FA02F1C2F1F1
:10313000200200FA02FC5FEA310040F1000053EA8D
:103140004C0308BF20EADC70704792F0000F00F0DB
:10315000004C02BF400010F4000F013AF9D040EAE1
:103160000C0093F0000F01F0004C02BF490011F475
:10317000000F013BF9D041EA0C018FE70CEAD15373
:1031800092EA0C0F18BF93EA0C0F0AD030F0004CF3
:1031900018BF31F0004CD8D180EA010000F00040A7
:1031A000704790F0000F17BF90F0004F084691F065
:1031B000000F91F0004F14D092EA0C0F01D142029F
:1031C0000FD193EA0C0F03D14B0218BF084608D168
:1031D00080EA010000F0004040F0FE4040F40000B2
:1031E000704740F0FE4040F4400070474FF0FF0C45
:1031F0001CEAD0521EBF1CEAD15392EA0C0F93EA8C
:103200000C0F69D0A2EB030280EA010C49024FEADD
:10321000402037D04FF0805343EA111143EA101396
:103220000CF000408B4238BF5B0042F17D024FF44E
:10323000000C8B4224BF5B1A40EA0C00B3EB510F29
:1032400024BFA3EB510340EA5C00B3EB910F24BF12
:10325000A3EB910340EA9C00B3EBD10F24BFA3EB97
:10326000D10340EADC001B0118BF5FEA1C1CE0D15F
:10327000FD2A3FF650AF8B4240EBC25008BF20F012
:10328000010070470CF0004C4CEA50207F32C2BF66
:10329000D2F1FF0340EAC250704740F400004FF003
:1032A0000003013A37E792F0000F00F0004C02BF34
:1032B000400010F4000F013AF9D040EA0C0093F0FE
:1032C000000F01F0004C02BF490011F4000F013B58
:1032D000F9D041EA0C0195E70CEAD15392EA0C0FC0
:1032E00008D142027FF47DAF93EA0C0F7FF470AFF8
:1032F000084676E793EA0C0F04D14B023FF44CAF3B
:1033000008466EE730F0004C18BF31F0004CCAD1CF
:1033100030F000427FF45CAF31F000437FF43CAF0B
:103320005FE700BF4FF0FF3C06E000BF4FF0010C2D
:1033300002E000BF4FF0010C4DF804CD4FEA40020F
:103340004FEA41037FEA226C18BF7FEA236C11D059
:1033500001B052EA530C18BF90EA010F58BFB2EB0C
:10336000030088BFC81738BF6FEAE17018BF40F08C
:10337000010070477FEA226C02D15FEA402C05D140
:103380007FEA236CE4D15FEA412CE1D05DF8040BC5
:10339000704700BF844608466146FFE70FB5FFF758
:1033A000C9FF002848BF10F1000F0FBD4DF808ED10
:1033B000FFF7F4FF0CBF012000205DF808FB00BF01
:1033C0004DF808EDFFF7EAFF34BF012000205DF85B
:1033D00008FB00BF4DF808EDFFF7E0FF94BF0120A8
:1033E00000205DF808FB00BF4DF808EDFFF7D2FFA5
:1033F00094BF012000205DF808FB00BF4DF808EDE8
:10340000FFF7C8FF34BF012000205DF808FB00BFB4
:103410004FEA4002B2F1FE4F0FD34FF09E03B3EBE1
:1034200012620DD94FEA002343F0004310F0004F21
:1034300023FA02F018BF404270474FF00000704777
:1034400012F1610F01D1420205D110F0004008BF16
:103450006FF0004070474FF00000704742000ED2FE
:10346000B2F1FE4F0BD34FF09E03B3EB126209D4BF
:103470004FEA002343F0004323FA02F070474FF075
:103480000000704712F1610F01D1420202D14FF0EA
:10349000FF3070474FF00000704700BF014B1868C5
:1034A000704700BF400000200A44914200F1FF3302
:1034B00000D1704710B511F8014B914203F8014F4C
:1034C000F9D110BD03460244934200D1704703F87E
:1034D000011BF9E7002B2DE9F0471E46BBBF03F1A6
:1034E00000431E4600232D2388B0149F144627F066
:1034F0002007129A462F109DDDF84CA0137004D0BF
:10350000452F00D10135022300E0032307AA0492CE
:1035100006AACDE902A2CDE900352246334600F0E5
:10352000E7FC472F804602D1119BDB0722D5462FAF
:1035300008EB050911D198F80030302B0AD1002290
:1035400000232046314602F025FC18B9C5F10105DB
:10355000CAF80050DAF800309944002200232046CF
:10356000314602F017FC08B1CDF81C903022079BC1
:103570004B4508D34046079B159AA3EB08031360FD
:1035800008B0BDE8F087591C07911A70EFE7F7B54E
:103590000029B6BF2D232B2349420929027043700D
:1035A00022DD0DF107031F460A2691FBF6F206FB0A
:1035B0001214632904F1300403F1FF3503F8014CC0
:1035C0000ADC303205F8012C023B821CBB42144657
:1035D00005D3201A03B0F0BD2B461146E5E713F8DA
:1035E000011B02F8011BF1E7302319448370041D0D
:1035F000C170EEE72DE9F04F91B00C461A9F93464B
:103600001E46054601F024FA03681846099300F0A7
:103610009FFB00230E933B680A90073323F00703B8
:1036200003F1080294F81880D4F800A03A60D3E9B6
:103630000023C4E91223D4E9127929F000430B9343
:103640004FF0FF32A84B38460B9902F0D5FB68BB10
:103650004FF0FF32A44B38460B9902F0AFFB28BB6A
:10366000002200233846494602F09EFB10B12D236C
:1036700084F843309D4F9E4BB8F1470F88BF1F46DB
:1036800003234FF0000923612AF00403236000960E
:103690005B460FAA2146284600F0CEF9013040F0E3
:1036A00093804FF0FF3011B0BDE8F08F3A464B46A3
:1036B0003846494602F0A0FB60B10022002338469C
:1036C000494602F071FB10B12D2384F84330894F35
:1036D000894BD1E7636808F0DF015A1C42D1062309
:1036E0006360002206920EAACDE904820DAA4AF474
:1036F000806303920DF13302CDE9013223606368E8
:103700003A46009328464B460B91FFF7E3FE0B9990
:10371000074647290D9908D1C81C02DB6368994206
:1037200040DDA8F102085FFA88F8B8F1650F1FD8EC
:103730000139424604F150000D91FFF728FF0E9A1F
:1037400081461318012A236102DC2268D20701D5C1
:10375000013323619DF83330002B98D02D2384F85A
:10376000433094E74729BCD1002BBAD10123B7E7F6
:10377000B8F1660F18D1002963680BDD216113B918
:103780002268D00702D501330B442361A1654FF0B5
:103790000009DFE713B92268D20701D50233F4E745
:1037A0000123F2E74FF067080E9B994205DB23687F
:1037B0002161D807EAD54B1CE7E70029CCBF0122DD
:1037C000C1F102021344E0E723685A0507D42369D4
:1037D0003A4659462846B047013029D161E7B8F149
:1037E000650F40F2D880D4E912010022002302F0D4
:1037F000D1FA88B30123414A59462846B0470130DF
:103800003FF44FAFDDE90D239A4202DB2368D8076E
:103810000ED5DDE9092359462846B04701303FF46B
:1038200040AF002704F11A080E9B013BBB4209DCA4
:1038300023689F0700F1FB80E0680F9B9842B8BFA8
:10384000184630E70123424659462846B047013022
:103850003FF427AF0137E7E70D9B002B2BDC01235B
:10386000264A59462846B04701303FF41AAFDDE9F1
:103870000D23134302D12368D907D9D5DDE90923E4
:1038800059462846B04701303FF40BAF4FF00008CF
:1038900004F11A090D9B5B42434501DC0E9B97E73F
:1038A00001234A4659462846B04701303FF4F9AE55
:1038B00008F10108EEE70E9AA36D9A42A8BF1A46D6
:1038C000002A904607DD134659463A462846B04737
:1038D00001303FF4E6AE04F11A034FF0000A28EA83
:1038E000E8780B9316E000BFFFFFEF7FD46100087C
:1038F000D8610008DC610008E0610008E4610008AC
:1039000001230B9A59462846B04701303FF4C9AE0F
:103910000AF1010AD4F85890A9EB08035345EFDCEB
:10392000DDE90D239A421ADB2368DA0717D4DDE9B3
:103930000D2391451BDBA3EB0908B8F1000F08DD4F
:10394000434607EB090259462846B04701303FF489
:10395000A8AE002728EAE87804F11A0913E0DDE9A7
:10396000092359462846B0470130E0D199E6A3EB38
:103970000208E2E701234A4659462846B04701308B
:103980003FF48FAE0137DDE90D239B1AA3EB08034B
:10399000BB42EFDC4CE70E9A012A01DCDB0734D591
:1039A00001233A4659462846B04701303FF479AEE4
:1039B000DDE9092359462846B04701303FF471AE8E
:1039C000D4E912010022002302F0E4F9C8B90E9BE9
:1039D0007A1C013B59462846B04701300DD160E6BC
:1039E0000123424659462846B04701303FF459AEBC
:1039F00001370E9B013BBB42F2DC4B4604F1500207
:103A0000E7E6002704F11A08F3E701233A46E1E765
:103A10000123424659462846B04701303FF441AEA3
:103A20000137E3680F9A9B1ABB42F1DC04E70027D9
:103A300004F11908F5E700BF2DE9F04791461F464C
:103A40008A680B6906469342B8BF1346C9F800302E
:103A500091F843200C46DDF8208012B10133C9F8FB
:103A600000302368990642BFD9F800300233C9F804
:103A70000030256815F0060507D104F1190AE3683E
:103A8000D9F800209B1AAB4229DC94F84330226815
:103A9000003318BF012392062ED404F143023946A5
:103AA0003046C047013021D02368E56803F00603A3
:103AB000042B18BF0025D9F800204FF0000908BFDB
:103AC000AD1AA368226908BF25EAE5759342C4BF11
:103AD0009B1AED181A344D451AD1002008E0012335
:103AE000524639463046C047013003D14FF0FF30CF
:103AF000BDE8F0870135C2E73020E11881F84300C6
:103B00005A1C94F845102244023382F84310C4E74B
:103B10000123224639463046C0470130E6D009F13C
:103B20000109D8E72DE9F04306460C4601F14300B0
:103B3000097E85B06E29984617460C9B00F0BB8025
:103B400024D8632939D00AD8002900F0C480582924
:103B500000F0928004F1420584F8421035E06429B7
:103B600001D06929F6D125681A6815F0800F02F195
:103B700004012CD012681960002A03DA2D23524266
:103B800084F84330DFF8C0C10A233FE0732900F016
:103B9000A68008D86F2921D07029DBD1226842F095
:103BA0002002226003E0752918D07829D2D178222A
:103BB000DFF898C184F8452062E01A6804F14205F4
:103BC000111D1960136884F84230012394E01268D3
:103BD00015F0400F196018BF12B2CDE7D4F800C03D
:103BE0001A681CF0800F02F104051D6001D01268F4
:103BF00003E01CF0400FFAD012886F290CBF082395
:103C00000A23DFF844C1002184F843106568002DC1
:103C1000A8BF2168A560A4BF21F0040121600AB9F2
:103C2000002D46D00546B2FBF3F103FB112E1CF824
:103C30000EE0934205F801ED39D9082B0BD123682A
:103C4000DA0708D5236962689A42DEBF302305F897
:103C5000013C05F1FF35401B2061CDF800803B465B
:103C600003AA21463046FFF7E7FE013049D14FF065
:103C7000FF3005B0BDE8F083DFF8CCC084F8451014
:103C80001D68216855F8042B1D600D060BD5CD0766
:103C900044BF41F0200121601AB9236823F02003BA
:103CA00023601023AFE74B0648BF92B2EFE70A4606
:103CB000B9E70546C1E71A68D4F800C0151D616967
:103CC0001CF0800F1D60136801D0196003E01CF028
:103CD000400FFAD01980002305462361BDE71A681A
:103CE000111D1960156800216268284600F0BCFEAD
:103CF00008B1401B606063682361002384F843308F
:103D0000ABE723692A4639463046C0470130AED07A
:103D100023689B0713D4E068039B9842B8BF1846FA
:103D2000A7E701234A4639463046C04701309ED0B6
:103D30000135E368039A9B1AAB42F2DCEBE70025FE
:103D400004F11909F5E700BFE6610008F761000812
:103D5000034613F8012B002AFBD1181A01387047CB
:103D600030B5141E05469BB0184605DA8B234FF07C
:103D7000FF302B601BB030BD4FF40273ADF80C3038
:103D80000CBF234604F1FF33029305934FF6FF73F4
:103D900000910491ADF80E3002461E9B69462846FC
:103DA00001F056FA431CBCBF8B232B60002CE1D0E2
:103DB0000022009B1A70DDE707B5009313460A4600
:103DC000014603480068FFF7CBFF03B05DF804FB32
:103DD000400000202DE9F74F03690C698046A3429B
:103DE000C0F28280013CA00008F1140501F1140723
:103DF0002B18019357F8243055F8242001339A42A8
:103E000007EB0009B2FBF3F632D34FF0000ABC46D1
:103E1000AE46D3465CF8042B93B206FB03A3120C08
:103E20004FEA134A06FB02A29BB2ABEB0303DEF898
:103E300000B04FEA124A1FFA8BFB5B441FFA82FB69
:103E4000DEF80020E145CBEB124202EB23429BB2AD
:103E500043EA02434FEA224B4EF8043BDAD22B5896
:103E600033B9019B043B9D421A4631D3C8F8104038
:103E7000404601F016F8002826DB28464FF0000CDB
:103E8000013657F8041BD0F800E08BB2ACEB03030B
:103E90001FFA8EF213440A0CC2EB1E4202EB2342BD
:103EA0009BB243EA0243B9454FEA224C40F8043B37
:103EB000E7D255F8242005EB84032AB9043B9D4240
:103EC0001A460BD3C8F81040304603B0BDE8F08F57
:103ED0001268043B002AC9D1013CC4E71268043BC4
:103EE000002AEFD1013CEAE70020EEE700000000E5
:103EF0002DE9F04F476A97B080461D46239E9246B3
:103F00009B4647B9102000F0A7FDC0E90177C8F82B
:103F100024000760C760D8F82430196859B15A687E
:103F2000012393404A608B60404600F0DFFD002291
:103F3000D8F824301A602B1EADBF0023012223F0D5
:103F4000004B3360AE4BB8BF326033EA0B035C46C4
:103F50001AD142F20F73229A1360CBF3130353EA80
:103F60000A0300F05F85249B53B9A64B21E0A64BC2
:103F700005930833249A1360059817B0BDE8F08FB5
:103F8000A04B05930333F5E7002200235046594622
:103F9000CDE90CAB01F0FEFE074660B10123229A89
:103FA0001360249B002B00F03A85984B249A1360F1
:103FB000013B0593E0E714AB019315AB009340463A
:103FC000DDE90C2300F0E5FFCBF30A560390002E49
:103FD00000F08180DDE90C450D9BA6F2FF36C3F3AE
:103FE000130343F07F5545F4401512970022884B88
:103FF0002046294601F0AEFA7BA3D3E9002301F065
:1040000061FC7BA3D3E9002301F0A6FA0446304605
:104010000D4601F0EDFB78A3D3E9002301F052FC3B
:1040200002460B462046294601F096FA04460D4604
:1040300001F0F8FE0022814600232046294601F0C7
:10404000B3FE48B1484601F0D3FB22462B4601F0AF
:10405000A1FE08B909F1FF39B9F1160F58D8DDE909
:104060000C016C4B03EBC903D3E9002301F09CFE68
:1040700000284FD0002309F1FF391193149B9E1B98
:10408000731E099345BFC6F1010308930023002363
:1040900054BF08930993B9F1000F3DDB099BCDF89C
:1040A00040904B44099300230A93209B092B00F274
:1040B0008D80052BC4BF043B2093209BC8BF0024E8
:1040C000A3F10203D8BF0124032B00F2A780DFE88D
:1040D00003F02D3A387BDDE914631E4406F23240CA
:1040E0002028C1BFC0F14000844006F212402AFAE5
:1040F00000F0D6BFC0F1200020430AFA00F001F022
:1041000067FB01230446A1F1F875013E12936DE7A8
:104110000123B2E71190B1E7089BA3EB09030893D1
:10412000C9F100030A9300231093BEE700230B9309
:10413000219B002B75DC01231A46069304932192E0
:104140000BE00123F3E700230B93219B4B440693E1
:104150000133012B0493B8BF01230022D8F8245067
:104160006A60042202F11400984269685DD94046F1
:1041700000F088FCD8F8243028601B680593049B65
:104180000E2B00F2D580002C00F0D280B9F1000F88
:1041900069DD204A09F00F0302EBC303D3E90034C1
:1041A000CDE90E344FEA2914E0065AD5DDE90C01B9
:1041B000194B0327D3E9082301F0AEFC82468B4656
:1041C00004F00F04144D41E00123BDE70124002356
:1041D0000B9420934FF0FF33002206930493122395
:1041E000ADE700BFAFF3008061436F63A787D23FA5
:1041F000B3C8608B288AC63FFB799F501344D33FD6
:104200000000F07F1162000808620008E561000804
:104210000000F83F406200081862000801230B9379
:10422000D8E7219B0693049397E701316960520018
:1042300098E7E10708D5DDE90E01D5E9002301F093
:1042400041FBCDE90E01013764100835002CF0D197
:10425000DDE90E235046594601F05EFC82468B464E
:104260001AE00227AEE700F09D80DDE90C01C9F1FC
:1042700000049B4B04F00F0203EBC203D3E90023BD
:1042800001F020FB022782468B460023954D241126
:10429000002C7CD1002BE1D1119B002B00F08480FD
:1042A0000022914B504659465D4601F07DFD0028A5
:1042B0007AD0049B002B77D0069B002B36DD50462E
:1042C00059460022894B01F0FDFA82468B46069C36
:1042D00009F1FF360137384601F08AFA52465B464B
:1042E00001F0F0FA0022824B01F036F9A1F150758D
:1042F000CDE90E010F95002C59D100227D4B50467F
:10430000594601F027F90E9A2B4682468B4601F05A
:1043100069FD002840F086820E9A05F10043504660
:10432000594601F041FD002840F07A82DDE90CABEE
:10433000159B002BC0F24B81B9F10E0F00F34781A2
:10434000674B03EBC903D3E90034CDE90634219B65
:10435000002B80F2D380049B002B00F3CF8040F031
:104360005E82DDE906010022624B01F0ABFA5246A3
:104370005B4601F02DFD049C2646002840F0378264
:104380003123059D09F1010905F8013B33E2E207FC
:1043900005D5D5E9002301F095FA01230137641012
:1043A000083575E7022777E74E46049C93E74C4BA8
:1043B00003EBC40353E90201059B1C440B9B002B38
:1043C00044D002460B4600204B4901F0A5FBDDE935
:1043D0000E2301F0BFF8CDE90E01059D5946504668
:1043E00001F020FD074601F003FA02460B46504655
:1043F000594601F0AFF8DDE90E23303705F8017BAF
:1044000082468B4601F0D0FC00285FD152465B46C5
:104410000020354901F09EF8DDE90E2301F0C4FCCF
:10442000002840F0B580A54280D0DDE90E010022D1
:104430002E4B01F047FA0022CDE90E012B4B5046DE
:10444000594601F03FFA82468B46C7E7DDE90E2365
:1044500001F038FA2546CDE90E01059F5946504630
:1044600001F0E0FC139001F0C3F902460B46504600
:10447000594601F06FF8139B8246303307F8013B31
:10448000A7428B464FF0000224D1DDE90E011A4B02
:1044900001F062F802460B465046594601F0A2FC74
:1044A000002875D1DDE90E230020134901F052F8F0
:1044B00002460B465046594601F076FC00283FF470
:1044C00035AF15F8013C6A1E302B01D0B1464EE0E5
:1044D0001546F6E7054B01F0F5F982468B46BDE738
:1044E00040620008186200080000F03F000024400D
:1044F00000001C40000014400000E03F56464FF012
:10450000000A5F46059DDFF844B5DDE90623304625
:10451000394601F001FB01F085FC044601F068F921
:10452000DDE9062301F0CEF902460B463046394656
:1045300001F010F804F1300605F8016B059E049FA8
:10454000AE1BB74202460B4634D101F005F8DDE957
:10455000062306460F4601F045FCC0B9DDE90623F7
:104560003046394601F016FC08B1E3070FD4039931
:10457000404600F0BBFA0023229A2B7009F1010398
:104580001360249B002B3FF4F7AC1D60F4E44E460F
:1045900015F8012C6B1E392A06D1059A9A4207D1CB
:1045A0003022059901360A701A7801321A708DE7A7
:1045B0001D46EDE752465B4601F084F900220023D8
:1045C00006460F4601F0E6FB00289ED0CFE70B9A87
:1045D000002A00F0CC80209A012A00F3AE80129AC3
:1045E000002A00F0A68003F233430A9C089D089A33
:1045F00001211A440892099A40461A44099200F08F
:1046000017FB0646002D0CDD099B002B09DDAB4294
:10461000A8BF2B46089AED1AD21A0892099AD31A03
:1046200009930A9BF3B10B9B002B00F0A480002C94
:1046300010DD31462246404600F092FB039A0146C7
:104640000646404600F0FDFA07460399404600F052
:104650004DFA03970A9B1A1B04D00399404600F0B9
:104660007FFB03900121404600F0E2FA109B0446D4
:10467000002B40F382801A460146404600F070FB52
:10468000209B0446012B7BDD0027236904EB830379
:10469000186900F07DFAC0F12000099B184410F061
:1046A0001F0000F08B80C0F12003042B40F38480B6
:1046B000C0F11C00089B054403440893099B034474
:1046C0000993089B002B05DD1A460399404600F02C
:1046D00095FB0390099B002B05DD21461A464046B9
:1046E00000F08CFB0446119B002B69D021460398F7
:1046F00000F0D7FB002863DA00230A220399404622
:1047000000F00BFA0B9B09F1FF390390002B00F02E
:104710009081002331460A22404600F0FEF9069BB4
:104720000646002B00F38780209B022B40F38380FA
:104730004EE0149BC3F1360357E7049B5C1E0A9BB3
:10474000A342B7BF0A9B1C1BE21A109BBEBF0A9470
:104750009B181093049BB8BF0024002BBBBF089B81
:10476000049A089D9D1AACBF049B00233FE70A9C56
:10477000089D0B9E46E70A9A6FE7209B012B17DCEA
:10478000BAF1000F14D1CBF313039BB92BF0004700
:104790003F0D3F0537B10127089B01330893099B63
:1047A00001330993109B002B7FF46FAF012074E756
:1047B0000027F7E75746F5E783D018461C3079E71E
:1047C000049B002B31DC209B022B2EDD049B0693E7
:1047D000069B63B921460522404600F09EF901463A
:1047E0000446039800F05DFB00283FF7C9AD219B0C
:1047F000059D6FEA030900272146404600F076F93F
:10480000002E3FF4B4AE2FB1B74203D03946404634
:1048100000F06CF93146404600F068F9A7E6002444
:104820002646E4E7B1462646AAE50B9B002B00F09E
:10483000BB80049B0693002D05DD31462A46404689
:1048400000F0DCFA0646002F52D07168404600F0B6
:1048500019F90546326906F10C01023292000C305A
:10486000FEF722FE01222946404600F0C7FA3746ED
:104870000646059B01330493DDE9052313440A939F
:104880000AF001030993049B2146039803F1FF3AC0
:10489000FFF7A0FA3946069000F1300B039800F0BC
:1048A00000FB324608902146404600F014FBC268E7
:1048B0000546FAB90146039800F0F3FA0246294684
:1048C00040460B9200F012F9209B0B9A049D43EA9C
:1048D0000201099B0B430FD1BBF1390F28D0089B74
:1048E000002B02DD069B03F1310B8AF800B083E751
:1048F0003046BCE70122E2E7089B002B04DB20994D
:104900000B4309990B431DD1002AEEDD01220399C7
:10491000404600F073FA2146039000F0C2FA0028E6
:1049200003DCE2D11BF0010FDFD0BBF1390FD9D18D
:1049300039238AF8003015F8013C6A1E392B63D000
:10494000013368E0002A07DDBBF1390FF0D00BF12D
:1049500001038AF800304FE7049B0A9A03F801BC70
:1049600093423AD000230A220399404600F0D5F83A
:10497000B74203904FF000034FF00A023946404619
:1049800007D100F0CAF807460646049B013304939A
:1049900079E700F0C2F83146074600230A22404674
:1049A00000F0BBF80646F0E7049B0693059D214600
:1049B0000398FFF70FFA059B00F1300B05F801BBD8
:1049C000EA1A069B934207DD00230A220399404618
:1049D00000F0A3F80390EAE700270122039940467C
:1049E00000F00CFA2146039000F05BFA0028A2DCEC
:1049F00002D11BF0010F9ED115F8013C6A1E302B2D
:104A00007FF4FAAE1546F7E7059B934205D13123B3
:104A1000059A09F101091370EEE615468BE7094B7B
:104A2000FFF7C7BA249B002B7FF4A1AA064BFFF720
:104A3000C0BA069B002BB9DC209B022B3FF7C8AE07
:104A4000B4E700BFE46100080862000800002440E9
:104A50000048704794010020024B0146186800F09E
:104A600041BB00BF4000002010B5C9B202449042D3
:104A7000034601D1002303E01C7801308C42F6D1BB
:104A8000184610BD70B5456A04460E463DB9102063
:104A9000FFF7E2FFC0E9015560620560C560656A25
:104AA000EB6883B1636ADB6853F82600B8B901216B
:104AB00001FA06F56A1D9200204600F0B8FA60B1CE
:104AC000C0E901650EE021220421204600F0AFFA82
:104AD000636AE860DB68002BE4D1002070BD0268E7
:104AE00043F826200023C0E90333F7E770B5446A92
:104AF00006460D463CB91020FFF7AEFFC0E9014461
:104B000070620460C4603DB1736A6A68DB6853F820
:104B10002210296043F8225070BD2DE9F0411F4654
:104B200006460C4600230D6901F1140CDCF8000068
:104B3000013381B202FB0171000C0F0C02FB00700B
:104B400089B201EB00419D424FEA10474CF8041B2B
:104B5000ECDCD7B1A368AB4212DC616830460131AE
:104B6000FFF790FF8046226904F10C0102329200A7
:104B70000C30FEF799FC21463046FFF7B7FF44465C
:104B800004EB850301355F6125612046BDE8F081B6
:104B9000020C12040346CAB90304102013F07F4F1D
:104BA00004BF1B02083013F0704F04BF1B01043018
:104BB00013F0404F04BF9B000230002B05DB13F0C5
:104BC000804F00F1010008BF202070470020E5E77A
:104BD0000368014613F007020BD0DA0724D49807C4
:104BE00049BF5B089B0801200B605CBF0B60022083
:104BF000704798B2B0B910201B0C13F0FF0F04BF20
:104C00001B0A08301A0704BF1B0904309A0704BFA7
:104C10009B080230DA0703D45B0800F1010005D0DD
:104C20000B6070471046E8E700207047202070476F
:104C300010B50C460121FFF725FF012244610261F6
:104C400010BD2DE9F74F90460A69D8F810300C4690
:104C50009A42BEBF0B46444698462769D8F8109042
:104C6000A368616807EB0906B342B8BF0131FFF7DB
:104C700009FF00F114052B46002205EB860E734553
:104C800016D304F1140308F1140203EB870702EBB7
:104C900089030093009B019293420CD8002E03DD00
:104CA0005EF8043D002B59D0066103B0BDE8F08FDB
:104CB00043F8042BE3E7B2F800A0BAF1000F23D0C9
:104CC000AC464FF0000804F1140959F8041BDCF855
:104CD00000B08BB21FFA8BFB0AFB03B34FEA114BF8
:104CE000DCF8001043444FEA11480AFB0B8101EB4A
:104CF00013419BB243EA01434F454FEA11484CF838
:104D0000043BE2D8CCF80080019B0432B3F8029057
:104D1000B9F1000F20D0AC464FF0000A2B6804F127
:104D20001408B8F80010BCF802B09BB209FB01B13E
:104D30008A4443EA0A434CF8043B58F8043BBCF865
:104D400000101B0C09FB0313474503EB1A434FEA02
:104D5000134AE6D8CCF8003004359BE7013E9DE7C6
:104D60002DE9F843154612F0030206460F4607D018
:104D7000214C013A002354F82220FFF7CEFE0746CB
:104D8000AD1035D0746A3CB91020FFF765FEC0E95C
:104D9000014470620460C460D6F82480D8F80840EA
:104DA0004CB940F271213046FFF742FF0023044620
:104DB000C8F8080003604FF00008EB070AD5394631
:104DC00022463046FFF73DFF814639463046FFF721
:104DD0008DFE4F466D100BD0206838B92246214613
:104DE0003046FFF72EFF2060C0F800800446E4E75D
:104DF0003846BDE8F88300BF086300082DE9F04796
:104E00000C460746164623694FEA621A0AEB030965
:104E10004968A36809F10105AB4233DB3846FFF767
:104E200031FE0023804600F1140100F11002184603
:104E300053452ADB20692AEAEA7A04F1140316F0C2
:104E40001F0201EB8A0103EB800C22D00020C2F18B
:104E5000200E1E689640304341F8040B53F8040BB3
:104E60009C4520FA0EF0F4D8086008B109F102055B
:104E7000013D3846C8F810502146FFF737FE40463E
:104E8000BDE8F08701315B00C6E742F8040F01334B
:104E9000CEE7043953F8042B9C4541F8042FF9D888
:104EA000E6E703690A6930B59B1A0CD19200143009
:104EB00014318418114454F8045D51F8042D9542BE
:104EC00003D005D30123184630BDA042F3D3FAE73F
:104ED0004FF0FF33F7E72DE9F0470D46074611463F
:104EE00028461446FFF7DDFF061E08D13146384636
:104EF000FFF7C8FD0123C0E90436BDE8F087A4BF71
:104F000023462C4638466168A6BF1D46002601266A
:104F1000FFF7B8FD4FF0000EC6602B69266904F15B
:104F2000140205F1140902EB860709EB830800F16E
:104F3000140152F804AB59F8045B1FFA8AF3734466
:104F4000ACB21B1B2C0CC4EB1A4404EB23449BB2E5
:104F50004FEA244EC84543EA0444944641F8044BC2
:104F6000E7D8BC4504D351F8043D83B10661C4E7DA
:104F70005CF8044BA2B27244131403EB144392B2D4
:104F800042EA03424FEA234E41F8042BE9E7013E8F
:104F9000E9E72DE9F3411C46DDE90865012190466A
:104FA000FFF770FDC4F31302C4F30A5407462CBB89
:104FB0000192B8F1000226D068460092FFF708FE81
:104FC0000099F0B1019AC0F1200302FA03F30B43F8
:104FD000C2407B610192019B002B14BF0221012181
:104FE000BB613961C4B1A4F2334404443460C0F1FC
:104FF00035002860384602B0BDE8F08142F48012E6
:10500000D6E77961E7E701A8FFF7E2FD0121019BFF
:1050100039617B612030E5E7A0F2324007EB810384
:1050200030601869FFF7B4FDC0EB4110E1E738B517
:1050300002FB01F4214600F055F8054618B122465E
:105040000021FEF73FFA284638BD000038B5054676
:10505000002943D051F8043C0C1F002BB8BFE418C2
:1050600000F02AFA1E4A1368104633B963601460D0
:105070002846BDE8384000F025BAA3420BD9216884
:105080006218934201BF1A685B685218226063601D
:105090000460EDE713465A680AB1A242FAD91968CA
:1050A0005818A0420BD12068014458188242196058
:1050B000DED110685268014419605A60D8E702D9FD
:1050C0000C232B60D4E7206821188A4201BF1168A5
:1050D00052680918216062605C60C9E738BD00BF92
:1050E000E8020020F8B5CD1C25F0030508350C2D8D
:1050F00038BF0C25002D064601DBA94203D90C233D
:1051000033600020F8BD00F0D7F921490A68144641
:105110009CB9204F3B6823B92146304600F090F9F6
:1051200038602946304600F08BF9431C23D10C230C
:105130003046336000F0C6F9E3E723685B1B17D401
:105140000B2B03D923601C44256004E06368A24252
:105150000CBF0B605360304600F0B4F904F10B0053
:10516000231D20F00700C21ACCD01B1AA350C9E798
:1051700022466468CCE7C41C24F00304A042E3D0B8
:10518000211A304600F05CF90130DDD1CFE700BFD5
:10519000E8020020EC0200202DE9F0478E688246EC
:1051A0009E420C469146984638D8B1F80CC01CF483
:1051B000906F31D062692568096902EB42026F1A6B
:1051C00002EBD272013355103B449D4238BF1D465D
:1051D0001CF4806F30D02946FFF784FF064650B993
:1051E0000C234FF0FF30CAF80030A38943F040038E
:1051F000A381BDE8F0873A462169FEF755F9A389F6
:1052000023F4906343F08003A38126613E4426602B
:1052100046466561ED1BA560464500D946463246C7
:105220004946206800F02EF9A36800209B1BA3606C
:1052300023681E442660DCE72A4600F049F906464A
:105240000028E2D121695046FFF700FFC8E70000BF
:105250002DE9F04F1E468B899DB01B0607460D4673
:1052600014460ED50B6963B94021FFF73BFF286058
:10527000286120B90C233B604FF0FF30C9E0402388
:105280006B610023099320238DF8293030234FF0E0
:10529000010ADFF898918DF82A30039623461E46BE
:1052A00013F8012B0AB1252AF9D1B6EB040B0BD068
:1052B0005B46224629463846FFF76EFF013000F074
:1052C000A380099B5B4409933378002B00F09C80FA
:1052D00000234FF0FF32CDE90523013604930793F5
:1052E0008DF853301A933446052214F8011B4F48A9
:1052F000FFF7BAFB049BC0B9D90644BF20228DF842
:1053000053201A0744BF2B228DF8532032782A2AC3
:1053100013D0344600200A26079A214611F8013B93
:10532000303B092B4BD970B914E0A0EB09000AFA05
:1053300000F0184304902646D5E7039A111D126821
:105340000391002A01DB079204E0524243F002037A
:105350000792049323782E2B0CD163782A2B33D118
:10536000039B02341A1D1B680392002BB8BF4FF039
:10537000FF3305932E4E032221783046FFF774FB4E
:1053800038B14023801B03FA00F0049B013403432F
:10539000049314F8011B062226488DF82810FFF705
:1053A00063FB002838D0244B13BB039B073323F047
:1053B000070308330393099B434409936EE706FBF5
:1053C000023201200C46A8E700230A2619460134C0
:1053D0000593204610F8012B303A092A03D9002BF7
:1053E000C8D00591C6E706FB012101230446F0E77A
:1053F00003AB00932A46114B04A93846FEF7FAF88E
:10540000B0F1FF3F8046D6D1AB895B063FF534AFA4
:1054100009981DB0BDE8F08F03AB00932A46074BF7
:1054200004A93846FEF77EFBEAE700BF14630008D4
:105430001A6300081E630008F5350008995100083A
:1054400038B50023054C054608462360FAF7FAFFF5
:10545000431C02D1236803B12B6038BDF002002049
:1054600082B001B901A942B14BB113780B60127837
:10547000101C18BF012002B070471046FBE76FF008
:105480000100F8E7884210B501EB020302D983421C
:105490001C4607D8421E994208D011F8014B02F869
:1054A000014FF8E783189A1A9A4200D110BD14F8F8
:1054B000011D03F8011DF7E7014800F03CB800BFEB
:1054C00094080020014800F037B800BF940800207D
:1054D000F8B5074614460E4621B91146BDE8F84016
:1054E000FFF700BE22B9FFF7B1FD25462846F8BDFB
:1054F00000F023F8A0420FD221463846FFF7F2FD14
:1055000005460028F2D031462246FDF7CDFF314650
:105510003846FFF79BFDE9E73546E7E749B1FF2A43
:105520008BBF8A230A700360012088BF4FF0FF30D1
:105530007047084670477047704751F8043C181F81
:10554000002BBCBF0B58C0187047000081F0004111
:1055500002E000BF83F0004330B54FEA41044FEA58
:10556000430594EA050F08BF90EA020F1FBF54EAF3
:10557000000C55EA020C7FEA645C7FEA655C00F08F
:10558000E2804FEA5454D4EB5555B8BF6D420CDD60
:105590002C4480EA020281EA030382EA000083EAE3
:1055A000010180EA020281EA0303362D88BF30BD83
:1055B00011F0004F4FEA01314FF4801C4CEA1131D9
:1055C00002D0404261EB410113F0004F4FEA033338
:1055D0004CEA133302D0524263EB430394EA050FC3
:1055E00000F0A780A4F10104D5F1200E0DDB02FA32
:1055F0000EFC22FA05F2801841F1000103FA0EF2C6
:10560000801843FA05F359410EE0A5F120050EF18B
:10561000200E012A03FA0EFC28BF4CF0020C43FABC
:1056200005F3C01851EBE37101F0004507D54FF0C9
:10563000000EDCF1000C7EEB00006EEB0101B1F519
:10564000801F1BD3B1F5001F0CD349085FEA30005F
:105650004FEA3C0C04F101044FEA445212F5800F6A
:1056600080F09A80BCF1004F08BF5FEA500C50F107
:10567000000041EB045141EA050130BD5FEA4C0CEA
:10568000404141EB010111F4801FA4F10104E9D173
:1056900091F0000F04BF01460020B1FA81F308BF6A
:1056A0002033A3F10B03B3F120020CDA0C3208DD36
:1056B00002F1140CC2F10C0201FA0CF021FA02F111
:1056C0000CE002F11402D8BFC2F1200C01FA02F181
:1056D00020FA0CFCDCBF41EA0C019040E41AA2BFA6
:1056E00001EB0451294330BD6FEA04041F3C1CDA6E
:1056F0000C340EDC04F11404C4F1200220FA04F08E
:1057000001FA02F340EA030021FA04F345EA030137
:1057100030BDC4F10C04C4F1200220FA02F001FAF9
:1057200004F340EA0300294630BD21FA04F029467B
:1057300030BD94F0000F83F4801306BF81F4801114
:105740000134013D4EE77FEA645C18BF7FEA655C87
:1057500029D094EA050F08BF90EA020F05D054EA59
:10576000000C04BF1946104630BD91EA030F1EBF5E
:105770000021002030BD5FEA545C05D14000494162
:1057800028BF41F0004130BD14F580043CBF01F555
:10579000801130BD01F0004545F0FE4141F470013B
:1057A0004FF0000030BD7FEA645C1ABF1946104616
:1057B0007FEA655C1CBF0B46024650EA013406BF17
:1057C00052EA033591EA030F41F4002130BD00BFD6
:1057D00090F0000F04BF0021704730B54FF4806493
:1057E00004F132044FF000054FF0000150E700BF14
:1057F00090F0000F04BF0021704730B54FF4806473
:1058000004F1320410F0004548BF40424FF000015F
:105810003EE700BF42004FEAE2014FEA31014FEAA2
:1058200002701FBF12F07F4393F07F4F81F06051F1
:10583000704732F07F4208BF704793F07F4F04BF3C
:1058400041F40021704730B54FF4607401F0004519
:1058500021F000411CE700BF50EA010208BF704779
:1058600030B54FF000050AE050EA010208BF70476A
:1058700030B511F0004502D5404261EB41014FF4D3
:10588000806404F132045FEA915C3FF4D8AE4FF0DB
:1058900003025FEADC0C18BF03325FEADC0C18BFBE
:1058A000033202EBDC02C2F1200300FA03FC20FA0F
:1058B00002F001FA03FE40EA0E0021FA02F114445C
:1058C000BDE600BF70B54FF0FF0C4CF4E06C1CEA75
:1058D00011541DBF1CEA135594EA0C0F95EA0C0FE6
:1058E00000F0DEF82C4481EA030621EA4C5123EA59
:1058F0004C5350EA013518BF52EA033541F4801188
:1059000043F4801338D0A0FB02CE4FF00005E1FB3A
:1059100002E506F00042E0FB03E54FF00006E1FB84
:1059200003569CF0000F18BF4EF0010EA4F1FF04C7
:10593000B6F5007F64F5407404D25FEA4E0E6D4107
:1059400046EB060642EAC62141EA55514FEAC52018
:1059500040EA5E504FEACE2EB4F1FD0C88BFBCF594
:10596000E06F1ED8BEF1004F08BF5FEA500E50F145
:10597000000041EB045170BD06F0004646EA01010B
:1059800040EA020081EA0301B4EB5C04C2BFD4EB3D
:105990000C0541EA045170BD41F480114FF0000E36
:1059A000013C00F3AB8014F1360FDEBF002001F0A4
:1059B000004170BDC4F10004203C35DA0C341BDC1E
:1059C00004F11404C4F1200500FA05F320FA04F0F0
:1059D00001FA05F240EA020001F0004221F0004124
:1059E00010EBD37021FA04F642EB06015EEA430E97
:1059F00008BF20EAD37070BDC4F10C04C4F12005C7
:105A000000FA04F320FA05F001FA04F240EA020079
:105A100001F0004110EBD37041F100015EEA430E4A
:105A200008BF20EAD37070BDC4F1200500FA05F26A
:105A30004EEA020E20FA04F301FA05F243EA0203E9
:105A400021FA04F001F0004121FA04F220EA0200F8
:105A500000EBD3705EEA430E08BF20EAD37070BD3E
:105A600094F0000F0FD101F00046400041EB01011E
:105A700011F4801F08BF013CF7D041EA060195F000
:105A8000000F18BF704703F00046520043EB0303BA
:105A900013F4801F08BF013DF7D043EA06037047A7
:105AA00094EA0C0F0CEA135518BF95EA0C0F0CD0B2
:105AB00050EA410618BF52EA4306D1D181EA0301F8
:105AC00001F000414FF0000070BD50EA410606BFF2
:105AD0001046194652EA430619D094EA0C0F02D137
:105AE00050EA013613D195EA0C0F05D152EA03367C
:105AF0001CBF104619460AD181EA030101F000419A
:105B000041F0FE4141F470014FF0000070BD41F0E2
:105B1000FE4141F4780170BD70B54FF0FF0C4CF4BC
:105B2000E06C1CEA11541DBF1CEA135594EA0C0FDB
:105B300095EA0C0F00F0A7F8A4EB050481EA030E28
:105B400052EA03354FEA013100F088804FEA03330F
:105B50004FF0805545EA131343EA12634FEA0222DD
:105B600045EA111545EA10654FEA00260EF000419E
:105B70009D4208BF964244F1FD0404F5407402D2F0
:105B80005B084FEA3202B61A65EB03055B084FEA81
:105B900032024FF480104FF4002CB6EB020E75EB7E
:105BA000030E22BFB61A754640EA0C005B084FEAA6
:105BB0003202B6EB020E75EB030E22BFB61A754623
:105BC00040EA5C005B084FEA3202B6EB020E75EB6E
:105BD000030E22BFB61A754640EA9C005B084FEAE6
:105BE0003202B6EB020E75EB030E22BFB61A7546F3
:105BF00040EADC0055EA060E18D04FEA051545EAE2
:105C000016754FEA06164FEAC30343EA52734FEA8A
:105C1000C2025FEA1C1CC0D111F4801F0BD141EA03
:105C200000014FF000004FF0004CB6E711F4801F68
:105C300004BF01430020B4F1FD0C88BFBCF5E06F48
:105C40003FF6AFAEB5EB030C04BFB6EB020C5FEA58
:105C5000500C50F1000041EB045170BD0EF0004EAD
:105C60004EEA113114EB5C04C2BFD4EB0C0541EADF
:105C7000045170BD41F480114FF0000E013C90E6DC
:105C800045EA060E8DE60CEA135594EA0C0F08BFA0
:105C900095EA0C0F3FF43BAF94EA0C0F0AD150EA9F
:105CA00001347FF434AF95EA0C0F7FF425AF104632
:105CB00019462CE795EA0C0F06D152EA03353FF45A
:105CC000FDAE1046194622E750EA410618BF52EAD7
:105CD00043067FF4C5AE50EA41047FF40DAF52EAAB
:105CE00043057FF4EBAE12E74FF0FF3C06E000BF48
:105CF0004FF0010C02E000BF4FF0010C4DF804CD55
:105D00004FEA410C7FEA6C5C4FEA430C18BF7FEA14
:105D10006C5C1BD001B050EA410C0CBF52EA430C42
:105D200091EA030F02BF90EA020F0020704710F1C2
:105D3000000F91EA030F58BF994208BF90422CBF51
:105D4000D8176FEAE37040F0010070474FEA410C4A
:105D50007FEA6C5C02D150EA013C07D14FEA430C68
:105D60007FEA6C5CD6D152EA033CD3D05DF8040BD9
:105D7000704700BF8446104662468C46194663460B
:105D800000E000BF01B5FFF7B7FF002848BF10F1E2
:105D9000000F01BD4DF808EDFFF7F4FF0CBF012027
:105DA00000205DF808FB00BF4DF808EDFFF7EAFFA3
:105DB00034BF012000205DF808FB00BF4DF808ED5E
:105DC000FFF7E0FF94BF012000205DF808FB00BF53
:105DD0004DF808EDFFF7CEFF94BF012000205DF8DD
:105DE00008FB00BF4DF808EDFFF7C4FF34BF0120EA
:105DF00000205DF808FB00BF4FEA410C7FEA6C5CB5
:105E000002D150EA013C0AD14FEA430C7FEA6C5CB4
:105E100002D152EA033C02D14FF0000070474FF02C
:105E2000010070474FEA410212F5001215D211D558
:105E30006FF47873B3EB625212D94FEAC12343F087
:105E4000004343EA505311F0004F23FA02F018BF09
:105E5000404270474FF00000704750EA013005D1D2
:105E600011F0004008BF6FF0004070474FF0000095
:105E7000704700BF537461636B206672616D653A51
:105E80000A000000205230203D2020253038580ADA
:105E900000000000205231203D2020253038580AD3
:105EA00000000000205232203D2020253038580AC2
:105EB00000000000205233203D2020253038580AB1
:105EC0000000000020523132203D20253038580A91
:105ED00000000000204C52203D2020253038580A78
:105EE00000000000205043203D2020253038580A73
:105EF0000000000020505352203D20253038580A21
:105F0000000000004653522F4641523A0A0000005A
:105F10002043465352203D2020253038580A0000A7
:105F20002048465352203D2020253038580A000092
:105F30002044465352203D2020253038580A000086
:105F40002041465352203D2020253038580A000079
:105F5000204D4D464152203D20253038580A000042
:105F60002042464152203D2020253038580A00006A
:105F70004D6973630A000000204C522F4558435F5F
:105F800052455455524E3D20253038580A000000E5
:105F90005B486172644661756C745D0A00000000C4
:105FA0005B4275734661756C745D0A005B55736185
:105FB00067654661756C745D0A00000000C1814030
:105FC00001C0804101C0804100C1814001C08041C9
:105FD00000C1814000C1814001C0804101C08041B9
:105FE00000C1814000C1814001C0804100C18140A9
:105FF00001C0804101C0804100C1814001C0804199
:1060000000C1814000C1814001C0804100C1814088
:1060100001C0804101C0804100C1814000C1814078
:1060200001C0804101C0804100C1814001C0804168
:1060300000C1814000C1814001C0804101C0804158
:1060400000C1814000C1814001C0804100C1814048
:1060500001C0804101C0804100C1814000C1814038
:1060600001C0804101C0804100C1814001C0804128
:1060700000C1814000C1814001C0804100C1814018
:1060800001C0804101C0804100C1814001C0804108
:1060900000C1814000C1814001C0804101C08041F8
:1060A00000C1814000C1814001C0804100C18140E8
:1060B00001C0804101C0804100C1814000C0C101D8
:1060C000C30302C2C60607C705C5C404CC0C0DCD68
:1060D0000FCFCE0E0ACACB0BC90908C8D81819D9D8
:1060E0001BDBDA1A1EDEDF1FDD1D1CDC14D4D51508
:1060F000D71716D6D21213D311D1D010F03031F1F8
:1061000033F3F23236F6F737F53534F43CFCFD3D27
:10611000FF3F3EFEFA3A3BFB39F9F83828E8E92917
:10612000EB2B2AEAEE2E2FEF2DEDEC2CE42425E5C7
:1061300027E7E62622E2E323E12120E0A06061A137
:1061400063A3A26266A6A767A56564A46CACAD6DE7
:10615000AF6F6EAEAA6A6BAB69A9A86878B8B97957
:10616000BB7B7ABABE7E7FBF7DBDBC7CB47475B587
:1061700077B7B67672B2B373B17170B05090915177
:106180009353529296565797559594549C5C5D9DA7
:106190005F9F9E5E5A9A9B5B995958988848498997
:1061A0004B8B8A4A4E8E8F4F8D4D4C8C4484854547
:1061B0008747468682424383418180405379737486
:1061C000656D20636C6F636B3A20257520487A0AF1
:1061D00000000000494E4600696E66004E414E00C8
:1061E0006E616E0030003031323334353637383935
:1061F0004142434445460030313233343536373836
:106200003961626364656600496E66696E697479B6
:10621000004E614E000000000080E03779C341432A
:10622000176E05B5B5B89346F5F93FE9034F384DFC
:10623000321D30F94877825A3CBF737FDD4F1575A8
:10624000000000000000F03F0000000000002440BB
:1062500000000000000059400000000000408F4096
:10626000000000000088C34000000000006AF84001
:106270000000000080842E4100000000D012634125
:106280000000000084D797410000000065CDCD419B
:10629000000000205FA00242000000E8764837427C
:1062A000000000A2941A6D42000040E59C30A2421A
:1062B0000000901EC4BCD64200003426F56B0C438F
:1062C0000080E03779C3414300A0D8855734764336
:1062D00000C84E676DC1AB43003D9160E458E14397
:1062E000408CB5781DAF154450EFE2D6E41A4B440C
:1062F00092D54D06CFF08044F64AE1C7022DB54451
:10630000B49DD9794378EA440500000019000000E3
:106310007D000000232D302B2000686C4C0065664A
:1063200067454647004300504F534958002E000030
:106330002020202020202020202828282828202035
:10634000202020202020202020202020202020204D
:1063500088101010101010101010101010101010C5
:1063600004040404040404040404101010101010A5
:10637000104141414141410101010101010101017E
:1063800001010101010101010101011010101010B2
:10639000104242424242420202020202020202024F
:1063A0000202020202020202020202101010102077
:1063B00000000000000000000000000000000000DD
:1063C00000000000000000000000000000000000CD
:1063D00000000000000000000000000000000000BD
:1063E00000000000000000000000000000000000AD
:1063F000000000000000000000000000000000009D
:10640000000000000000000000000000000000008C
:10641000000000000000000000000000000000007C
:10642000000000000000000000000000000000006C
:10643000785634121C02002000000000000000000A
:1064400000000000010203040607080900366E017F
:10645000010000000400000003000000E803000049
:10646000320000000100FFFF0100000014000000E6
:1064700044000020000000000000000000000000B8
:10648000000000000000000000000000000000000C
:1064900000000000000000000000000000000000FC
:1064A00000000000000000000000000000000000EC
:1064B00000000000000000000000000000000000DC
:1064C00000000000000000000000000000000000CC
:1064D0000000000043000000000000000000000079
:1064E00000000000000000000000000000000000AC
:1064F0000000000043000000000000000000000059
:10650000000000000000000000000000000000008B
:106510000000000043000000000000000000000038
:10652000000000000000000000000000000000006B
:106530000000000043000000000000000000000018
:10654000000000000000000000000000000000004B
:1065500000000000430000000000000000000000F8
:10656000000000000000000000000000000000002B
:1065700000000000430000000000000000000000D8
:10658000000000000000000000000000000000000B
:1065900000000000430000000000000000000000B8
:1065A00000000000000000000000000000000000EB
:1065B000000000001D5500086154000800000000A4
:1065C0002F6300082D630008196300081963000891
:1065D00019630008196300081963000819630008AB
:1065E000196300081963000819630008FFFFFFFF23
:1065F000FFFFFFFFFFFFFFFFFFFF00000100415310
:1066000043494900000000000000000000000000B5
:1066100000000000000000000000000000004153E6
:106620004349490000000000000000000000000095
:10663000000000000000000000000000000000005A
:0466400032547698C2
:04000005080001D11D
:00000001FF
